 Iex_dll

 Timestamp is 44d97f4d (Tue Aug 08 23:23:09 2006)

 Preferred load address is 10000000

 Start         Length     Name                   Class
 0001:00000000 00002a96H .text                   CODE
 0001:00002aa0 0000009aH .text$x                 CODE
 0002:00000000 00000108H .idata$5                DATA
 0002:00000108 00000004H .CRT$XCA                DATA
 0002:0000010c 00000004H .CRT$XCZ                DATA
 0002:00000110 00000004H .CRT$XIA                DATA
 0002:00000114 00000004H .CRT$XIAA               DATA
 0002:00000118 00000004H .CRT$XIZ                DATA
 0002:00000120 00000800H .rdata                  DATA
 0002:00000920 00001168H .rdata$r                DATA
 0002:00001a90 00000010H .rdata$sxdata           DATA
 0002:00001aa0 00000004H .rtc$IAA                DATA
 0002:00001aa4 00000000H .rtc$IMZ                DATA
 0002:00001aa4 00000004H .rtc$IZZ                DATA
 0002:00001aa8 00000004H .rtc$TAA                DATA
 0002:00001aac 00000000H .rtc$TMZ                DATA
 0002:00001aac 00000004H .rtc$TZZ                DATA
 0002:00001ab0 00000e3cH .xdata$x                DATA
 0002:000028ec 0000003cH .idata$2                DATA
 0002:00002928 00000014H .idata$3                DATA
 0002:0000293c 00000108H .idata$4                DATA
 0002:00002a44 00000796H .idata$6                DATA
 0002:000031da 00000000H .edata                  DATA
 0003:00000000 000005d0H .data                   DATA
 0003:000005d0 00000368H .bss                    DATA

  Address         Publics by Value              Rva+Base       Lib:Object

 0000:00000004       ___safe_se_handler_count   00000004     <absolute>
 0000:00000000       ___ImageBase               10000000     <linker-defined>
 0001:00000000       ?setStackTracer@Iex@@YAXP6A?AV?$basic_string@DU?$char_traits@D@std@@V?$allocator@D@2@@std@@XZ@Z 10001000 f   IexBaseExc.obj
 0001:00000010       ?stackTracer@Iex@@YAP6A?AV?$basic_string@DU?$char_traits@D@std@@V?$allocator@D@2@@std@@XZXZ 10001010 f   IexBaseExc.obj
 0001:00000020       ??0BaseExc@Iex@@QAE@PBD@Z  10001020 f   IexBaseExc.obj
 0001:00000150       ??0BaseExc@Iex@@QAE@ABV?$basic_string@DU?$char_traits@D@std@@V?$allocator@D@2@@std@@@Z 10001150 f   IexBaseExc.obj
 0001:00000260       ??0BaseExc@Iex@@QAE@AAV?$basic_stringstream@DU?$char_traits@D@std@@V?$allocator@D@2@@std@@@Z 10001260 f   IexBaseExc.obj
 0001:00000370       ??0BaseExc@Iex@@QAE@ABV01@@Z 10001370 f   IexBaseExc.obj
 0001:00000410       ??1BaseExc@Iex@@UAE@XZ     10001410 f   IexBaseExc.obj
 0001:000004a0       ?what@BaseExc@Iex@@UBEPBDXZ 100014a0 f   IexBaseExc.obj
 0001:000004e0       ?assign@BaseExc@Iex@@QAEAAV12@AAV?$basic_stringstream@DU?$char_traits@D@std@@V?$allocator@D@2@@std@@@Z 100014e0 f   IexBaseExc.obj
 0001:000005a0       ?append@BaseExc@Iex@@QAEAAV12@AAV?$basic_stringstream@DU?$char_traits@D@std@@V?$allocator@D@2@@std@@@Z 100015a0 f   IexBaseExc.obj
 0001:00000660       ?throwErrnoExc@Iex@@YAXABV?$basic_string@DU?$char_traits@D@std@@V?$allocator@D@2@@std@@H@Z 10001660 f   IexThrowErrnoExc.obj
 0001:00000f10       ?throwErrnoExc@Iex@@YAXABV?$basic_string@DU?$char_traits@D@std@@V?$allocator@D@2@@std@@@Z 10001f10 f   IexThrowErrnoExc.obj
 0001:00000f40       ??0ErrnoExc@Iex@@QAE@ABV?$basic_string@DU?$char_traits@D@std@@V?$allocator@D@2@@std@@@Z 10001f40 f i IexThrowErrnoExc.obj
 0001:00000f80       ??1EexistExc@Iex@@UAE@XZ   10001f80 f i IexThrowErrnoExc.obj
 0001:00000f80       ??1EnxioExc@Iex@@UAE@XZ    10001f80 f i IexThrowErrnoExc.obj
 0001:00000f80       ??1EpermExc@Iex@@UAE@XZ    10001f80 f i IexThrowErrnoExc.obj
 0001:00000f80       ??1EdomExc@Iex@@UAE@XZ     10001f80 f i IexThrowErrnoExc.obj
 0001:00000f80       ??1E2bigExc@Iex@@UAE@XZ    10001f80 f i IexThrowErrnoExc.obj
 0001:00000f80       ??1ErangeExc@Iex@@UAE@XZ   10001f80 f i IexThrowErrnoExc.obj
 0001:00000f80       ??1EmlinkExc@Iex@@UAE@XZ   10001f80 f i IexThrowErrnoExc.obj
 0001:00000f80       ??1EbusyExc@Iex@@UAE@XZ    10001f80 f i IexThrowErrnoExc.obj
 0001:00000f80       ??1EilseqExc@Iex@@UAE@XZ   10001f80 f i IexThrowErrnoExc.obj
 0001:00000f80       ??1EnomemExc@Iex@@UAE@XZ   10001f80 f i IexThrowErrnoExc.obj
 0001:00000f80       ??1EnoentExc@Iex@@UAE@XZ   10001f80 f i IexThrowErrnoExc.obj
 0001:00000f80       ??1EmfileExc@Iex@@UAE@XZ   10001f80 f i IexThrowErrnoExc.obj
 0001:00000f80       ??1EfbigExc@Iex@@UAE@XZ    10001f80 f i IexThrowErrnoExc.obj
 0001:00000f80       ??1EsrchExc@Iex@@UAE@XZ    10001f80 f i IexThrowErrnoExc.obj
 0001:00000f80       ??1EnotemptyExc@Iex@@UAE@XZ 10001f80 f i IexThrowErrnoExc.obj
 0001:00000f80       ??1ExdevExc@Iex@@UAE@XZ    10001f80 f i IexThrowErrnoExc.obj
 0001:00000f80       ??1EnottyExc@Iex@@UAE@XZ   10001f80 f i IexThrowErrnoExc.obj
 0001:00000f80       ??1EnospcExc@Iex@@UAE@XZ   10001f80 f i IexThrowErrnoExc.obj
 0001:00000f80       ??1EnosysExc@Iex@@UAE@XZ   10001f80 f i IexThrowErrnoExc.obj
 0001:00000f80       ??1EnfileExc@Iex@@UAE@XZ   10001f80 f i IexThrowErrnoExc.obj
 0001:00000f80       ??1EnametoolongExc@Iex@@UAE@XZ 10001f80 f i IexThrowErrnoExc.obj
 0001:00000f80       ??1EagainExc@Iex@@UAE@XZ   10001f80 f i IexThrowErrnoExc.obj
 0001:00000f80       ??1EnoexecExc@Iex@@UAE@XZ  10001f80 f i IexThrowErrnoExc.obj
 0001:00000f80       ??1EbadfExc@Iex@@UAE@XZ    10001f80 f i IexThrowErrnoExc.obj
 0001:00000f80       ??1EioExc@Iex@@UAE@XZ      10001f80 f i IexThrowErrnoExc.obj
 0001:00000f80       ??1EspipeExc@Iex@@UAE@XZ   10001f80 f i IexThrowErrnoExc.obj
 0001:00000f80       ??1EinvalExc@Iex@@UAE@XZ   10001f80 f i IexThrowErrnoExc.obj
 0001:00000f80       ??1EdeadlkExc@Iex@@UAE@XZ  10001f80 f i IexThrowErrnoExc.obj
 0001:00000f80       ??1EisdirExc@Iex@@UAE@XZ   10001f80 f i IexThrowErrnoExc.obj
 0001:00000f80       ??1EintrExc@Iex@@UAE@XZ    10001f80 f i IexThrowErrnoExc.obj
 0001:00000f80       ??1EaccesExc@Iex@@UAE@XZ   10001f80 f i IexThrowErrnoExc.obj
 0001:00000f80       ??1EpipeExc@Iex@@UAE@XZ    10001f80 f i IexThrowErrnoExc.obj
 0001:00000f80       ??1EnotdirExc@Iex@@UAE@XZ  10001f80 f i IexThrowErrnoExc.obj
 0001:00000f80       ??1ErofsExc@Iex@@UAE@XZ    10001f80 f i IexThrowErrnoExc.obj
 0001:00000f80       ??1EnodevExc@Iex@@UAE@XZ   10001f80 f i IexThrowErrnoExc.obj
 0001:00000f80       ??1EfaultExc@Iex@@UAE@XZ   10001f80 f i IexThrowErrnoExc.obj
 0001:00000f80       ??1ErrnoExc@Iex@@UAE@XZ    10001f80 f i IexThrowErrnoExc.obj
 0001:00000f80       ??1EnolckExc@Iex@@UAE@XZ   10001f80 f i IexThrowErrnoExc.obj
 0001:00000f80       ??1EchildExc@Iex@@UAE@XZ   10001f80 f i IexThrowErrnoExc.obj
 0001:00000fb0       ??_GEfbigExc@Iex@@UAEPAXI@Z 10001fb0 f i IexThrowErrnoExc.obj
 0001:00000fb0       ??_GEnosysExc@Iex@@UAEPAXI@Z 10001fb0 f i IexThrowErrnoExc.obj
 0001:00000fb0       ??_EExdevExc@Iex@@UAEPAXI@Z 10001fb0 f i IexThrowErrnoExc.obj
 0001:00000fb0       ??_GEdomExc@Iex@@UAEPAXI@Z 10001fb0 f i IexThrowErrnoExc.obj
 0001:00000fb0       ??_EEaccesExc@Iex@@UAEPAXI@Z 10001fb0 f i IexThrowErrnoExc.obj
 0001:00000fb0       ??_GEbadfExc@Iex@@UAEPAXI@Z 10001fb0 f i IexThrowErrnoExc.obj
 0001:00000fb0       ??_EEsrchExc@Iex@@UAEPAXI@Z 10001fb0 f i IexThrowErrnoExc.obj
 0001:00000fb0       ??_GErrnoExc@Iex@@UAEPAXI@Z 10001fb0 f i IexThrowErrnoExc.obj
 0001:00000fb0       ??_GEnfileExc@Iex@@UAEPAXI@Z 10001fb0 f i IexThrowErrnoExc.obj
 0001:00000fb0       ??_GEnomemExc@Iex@@UAEPAXI@Z 10001fb0 f i IexThrowErrnoExc.obj
 0001:00000fb0       ??_EEisdirExc@Iex@@UAEPAXI@Z 10001fb0 f i IexThrowErrnoExc.obj
 0001:00000fb0       ??_EEpipeExc@Iex@@UAEPAXI@Z 10001fb0 f i IexThrowErrnoExc.obj
 0001:00000fb0       ??_GEchildExc@Iex@@UAEPAXI@Z 10001fb0 f i IexThrowErrnoExc.obj
 0001:00000fb0       ??_EErangeExc@Iex@@UAEPAXI@Z 10001fb0 f i IexThrowErrnoExc.obj
 0001:00000fb0       ??_EEnolckExc@Iex@@UAEPAXI@Z 10001fb0 f i IexThrowErrnoExc.obj
 0001:00000fb0       ??_EEnoexecExc@Iex@@UAEPAXI@Z 10001fb0 f i IexThrowErrnoExc.obj
 0001:00000fb0       ??_EEagainExc@Iex@@UAEPAXI@Z 10001fb0 f i IexThrowErrnoExc.obj
 0001:00000fb0       ??_GEfaultExc@Iex@@UAEPAXI@Z 10001fb0 f i IexThrowErrnoExc.obj
 0001:00000fb0       ??_EE2bigExc@Iex@@UAEPAXI@Z 10001fb0 f i IexThrowErrnoExc.obj
 0001:00000fb0       ??_GEnoentExc@Iex@@UAEPAXI@Z 10001fb0 f i IexThrowErrnoExc.obj
 0001:00000fb0       ??_EEexistExc@Iex@@UAEPAXI@Z 10001fb0 f i IexThrowErrnoExc.obj
 0001:00000fb0       ??_EBaseExc@Iex@@UAEPAXI@Z 10001fb0 f i IexBaseExc.obj
 0001:00000fb0       ??_GExdevExc@Iex@@UAEPAXI@Z 10001fb0 f i IexThrowErrnoExc.obj
 0001:00000fb0       ??_EEchildExc@Iex@@UAEPAXI@Z 10001fb0 f i IexThrowErrnoExc.obj
 0001:00000fb0       ??_EEnametoolongExc@Iex@@UAEPAXI@Z 10001fb0 f i IexThrowErrnoExc.obj
 0001:00000fb0       ??_EEintrExc@Iex@@UAEPAXI@Z 10001fb0 f i IexThrowErrnoExc.obj
 0001:00000fb0       ??_GEaccesExc@Iex@@UAEPAXI@Z 10001fb0 f i IexThrowErrnoExc.obj
 0001:00000fb0       ??_EEmfileExc@Iex@@UAEPAXI@Z 10001fb0 f i IexThrowErrnoExc.obj
 0001:00000fb0       ??_GEnotemptyExc@Iex@@UAEPAXI@Z 10001fb0 f i IexThrowErrnoExc.obj
 0001:00000fb0       ??_GE2bigExc@Iex@@UAEPAXI@Z 10001fb0 f i IexThrowErrnoExc.obj
 0001:00000fb0       ??_EEilseqExc@Iex@@UAEPAXI@Z 10001fb0 f i IexThrowErrnoExc.obj
 0001:00000fb0       ??_EEnottyExc@Iex@@UAEPAXI@Z 10001fb0 f i IexThrowErrnoExc.obj
 0001:00000fb0       ??_EEnosysExc@Iex@@UAEPAXI@Z 10001fb0 f i IexThrowErrnoExc.obj
 0001:00000fb0       ??_GEbusyExc@Iex@@UAEPAXI@Z 10001fb0 f i IexThrowErrnoExc.obj
 0001:00000fb0       ??_GEmlinkExc@Iex@@UAEPAXI@Z 10001fb0 f i IexThrowErrnoExc.obj
 0001:00000fb0       ??_GEisdirExc@Iex@@UAEPAXI@Z 10001fb0 f i IexThrowErrnoExc.obj
 0001:00000fb0       ??_EEnoentExc@Iex@@UAEPAXI@Z 10001fb0 f i IexThrowErrnoExc.obj
 0001:00000fb0       ??_GEnodevExc@Iex@@UAEPAXI@Z 10001fb0 f i IexThrowErrnoExc.obj
 0001:00000fb0       ??_EEdeadlkExc@Iex@@UAEPAXI@Z 10001fb0 f i IexThrowErrnoExc.obj
 0001:00000fb0       ??_GErangeExc@Iex@@UAEPAXI@Z 10001fb0 f i IexThrowErrnoExc.obj
 0001:00000fb0       ??_GEnoexecExc@Iex@@UAEPAXI@Z 10001fb0 f i IexThrowErrnoExc.obj
 0001:00000fb0       ??_EEnospcExc@Iex@@UAEPAXI@Z 10001fb0 f i IexThrowErrnoExc.obj
 0001:00000fb0       ??_GEnospcExc@Iex@@UAEPAXI@Z 10001fb0 f i IexThrowErrnoExc.obj
 0001:00000fb0       ??_EEdomExc@Iex@@UAEPAXI@Z 10001fb0 f i IexThrowErrnoExc.obj
 0001:00000fb0       ??_EEspipeExc@Iex@@UAEPAXI@Z 10001fb0 f i IexThrowErrnoExc.obj
 0001:00000fb0       ??_EEfaultExc@Iex@@UAEPAXI@Z 10001fb0 f i IexThrowErrnoExc.obj
 0001:00000fb0       ??_GEpipeExc@Iex@@UAEPAXI@Z 10001fb0 f i IexThrowErrnoExc.obj
 0001:00000fb0       ??_GEinvalExc@Iex@@UAEPAXI@Z 10001fb0 f i IexThrowErrnoExc.obj
 0001:00000fb0       ??_EEnotdirExc@Iex@@UAEPAXI@Z 10001fb0 f i IexThrowErrnoExc.obj
 0001:00000fb0       ??_GBaseExc@Iex@@UAEPAXI@Z 10001fb0 f i IexBaseExc.obj
 0001:00000fb0       ??_EEbusyExc@Iex@@UAEPAXI@Z 10001fb0 f i IexThrowErrnoExc.obj
 0001:00000fb0       ??_EEinvalExc@Iex@@UAEPAXI@Z 10001fb0 f i IexThrowErrnoExc.obj
 0001:00000fb0       ??_EEbadfExc@Iex@@UAEPAXI@Z 10001fb0 f i IexThrowErrnoExc.obj
 0001:00000fb0       ??_GEnotdirExc@Iex@@UAEPAXI@Z 10001fb0 f i IexThrowErrnoExc.obj
 0001:00000fb0       ??_GEnolckExc@Iex@@UAEPAXI@Z 10001fb0 f i IexThrowErrnoExc.obj
 0001:00000fb0       ??_GErofsExc@Iex@@UAEPAXI@Z 10001fb0 f i IexThrowErrnoExc.obj
 0001:00000fb0       ??_EEnomemExc@Iex@@UAEPAXI@Z 10001fb0 f i IexThrowErrnoExc.obj
 0001:00000fb0       ??_EErofsExc@Iex@@UAEPAXI@Z 10001fb0 f i IexThrowErrnoExc.obj
 0001:00000fb0       ??_GEmfileExc@Iex@@UAEPAXI@Z 10001fb0 f i IexThrowErrnoExc.obj
 0001:00000fb0       ??_EEpermExc@Iex@@UAEPAXI@Z 10001fb0 f i IexThrowErrnoExc.obj
 0001:00000fb0       ??_EEfbigExc@Iex@@UAEPAXI@Z 10001fb0 f i IexThrowErrnoExc.obj
 0001:00000fb0       ??_GEioExc@Iex@@UAEPAXI@Z  10001fb0 f i IexThrowErrnoExc.obj
 0001:00000fb0       ??_GEsrchExc@Iex@@UAEPAXI@Z 10001fb0 f i IexThrowErrnoExc.obj
 0001:00000fb0       ??_GEexistExc@Iex@@UAEPAXI@Z 10001fb0 f i IexThrowErrnoExc.obj
 0001:00000fb0       ??_EEnfileExc@Iex@@UAEPAXI@Z 10001fb0 f i IexThrowErrnoExc.obj
 0001:00000fb0       ??_EEioExc@Iex@@UAEPAXI@Z  10001fb0 f i IexThrowErrnoExc.obj
 0001:00000fb0       ??_GEpermExc@Iex@@UAEPAXI@Z 10001fb0 f i IexThrowErrnoExc.obj
 0001:00000fb0       ??_GEilseqExc@Iex@@UAEPAXI@Z 10001fb0 f i IexThrowErrnoExc.obj
 0001:00000fb0       ??_EEnotemptyExc@Iex@@UAEPAXI@Z 10001fb0 f i IexThrowErrnoExc.obj
 0001:00000fb0       ??_GEdeadlkExc@Iex@@UAEPAXI@Z 10001fb0 f i IexThrowErrnoExc.obj
 0001:00000fb0       ??_EEnodevExc@Iex@@UAEPAXI@Z 10001fb0 f i IexThrowErrnoExc.obj
 0001:00000fb0       ??_GEintrExc@Iex@@UAEPAXI@Z 10001fb0 f i IexThrowErrnoExc.obj
 0001:00000fb0       ??_GEspipeExc@Iex@@UAEPAXI@Z 10001fb0 f i IexThrowErrnoExc.obj
 0001:00000fb0       ??_EErrnoExc@Iex@@UAEPAXI@Z 10001fb0 f i IexThrowErrnoExc.obj
 0001:00000fb0       ??_GEnottyExc@Iex@@UAEPAXI@Z 10001fb0 f i IexThrowErrnoExc.obj
 0001:00000fb0       ??_EEnxioExc@Iex@@UAEPAXI@Z 10001fb0 f i IexThrowErrnoExc.obj
 0001:00000fb0       ??_EEmlinkExc@Iex@@UAEPAXI@Z 10001fb0 f i IexThrowErrnoExc.obj
 0001:00000fb0       ??_GEagainExc@Iex@@UAEPAXI@Z 10001fb0 f i IexThrowErrnoExc.obj
 0001:00000fb0       ??_GEnametoolongExc@Iex@@UAEPAXI@Z 10001fb0 f i IexThrowErrnoExc.obj
 0001:00000fb0       ??_GEnxioExc@Iex@@UAEPAXI@Z 10001fb0 f i IexThrowErrnoExc.obj
 0001:00000ff0       ??0EpermExc@Iex@@QAE@ABV01@@Z 10001ff0 f i IexThrowErrnoExc.obj
 0001:00001030       ??0ErrnoExc@Iex@@QAE@ABV01@@Z 10002030 f i IexThrowErrnoExc.obj
 0001:00001070       ??0EnoentExc@Iex@@QAE@ABV01@@Z 10002070 f i IexThrowErrnoExc.obj
 0001:000010b0       ??0EsrchExc@Iex@@QAE@ABV01@@Z 100020b0 f i IexThrowErrnoExc.obj
 0001:000010f0       ??0EintrExc@Iex@@QAE@ABV01@@Z 100020f0 f i IexThrowErrnoExc.obj
 0001:00001130       ??0EioExc@Iex@@QAE@ABV01@@Z 10002130 f i IexThrowErrnoExc.obj
 0001:00001170       ??0EnxioExc@Iex@@QAE@ABV01@@Z 10002170 f i IexThrowErrnoExc.obj
 0001:000011b0       ??0E2bigExc@Iex@@QAE@ABV01@@Z 100021b0 f i IexThrowErrnoExc.obj
 0001:000011f0       ??0EnoexecExc@Iex@@QAE@ABV01@@Z 100021f0 f i IexThrowErrnoExc.obj
 0001:00001230       ??0EbadfExc@Iex@@QAE@ABV01@@Z 10002230 f i IexThrowErrnoExc.obj
 0001:00001270       ??0EchildExc@Iex@@QAE@ABV01@@Z 10002270 f i IexThrowErrnoExc.obj
 0001:000012b0       ??0EagainExc@Iex@@QAE@ABV01@@Z 100022b0 f i IexThrowErrnoExc.obj
 0001:000012f0       ??0EnomemExc@Iex@@QAE@ABV01@@Z 100022f0 f i IexThrowErrnoExc.obj
 0001:00001330       ??0EaccesExc@Iex@@QAE@ABV01@@Z 10002330 f i IexThrowErrnoExc.obj
 0001:00001370       ??0EfaultExc@Iex@@QAE@ABV01@@Z 10002370 f i IexThrowErrnoExc.obj
 0001:000013b0       ??0EbusyExc@Iex@@QAE@ABV01@@Z 100023b0 f i IexThrowErrnoExc.obj
 0001:000013f0       ??0EexistExc@Iex@@QAE@ABV01@@Z 100023f0 f i IexThrowErrnoExc.obj
 0001:00001430       ??0ExdevExc@Iex@@QAE@ABV01@@Z 10002430 f i IexThrowErrnoExc.obj
 0001:00001470       ??0EnodevExc@Iex@@QAE@ABV01@@Z 10002470 f i IexThrowErrnoExc.obj
 0001:000014b0       ??0EnotdirExc@Iex@@QAE@ABV01@@Z 100024b0 f i IexThrowErrnoExc.obj
 0001:000014f0       ??0EisdirExc@Iex@@QAE@ABV01@@Z 100024f0 f i IexThrowErrnoExc.obj
 0001:00001530       ??0EinvalExc@Iex@@QAE@ABV01@@Z 10002530 f i IexThrowErrnoExc.obj
 0001:00001570       ??0EnfileExc@Iex@@QAE@ABV01@@Z 10002570 f i IexThrowErrnoExc.obj
 0001:000015b0       ??0EmfileExc@Iex@@QAE@ABV01@@Z 100025b0 f i IexThrowErrnoExc.obj
 0001:000015f0       ??0EnottyExc@Iex@@QAE@ABV01@@Z 100025f0 f i IexThrowErrnoExc.obj
 0001:00001630       ??0EfbigExc@Iex@@QAE@ABV01@@Z 10002630 f i IexThrowErrnoExc.obj
 0001:00001670       ??0EnospcExc@Iex@@QAE@ABV01@@Z 10002670 f i IexThrowErrnoExc.obj
 0001:000016b0       ??0EspipeExc@Iex@@QAE@ABV01@@Z 100026b0 f i IexThrowErrnoExc.obj
 0001:000016f0       ??0ErofsExc@Iex@@QAE@ABV01@@Z 100026f0 f i IexThrowErrnoExc.obj
 0001:00001730       ??0EmlinkExc@Iex@@QAE@ABV01@@Z 10002730 f i IexThrowErrnoExc.obj
 0001:00001770       ??0EpipeExc@Iex@@QAE@ABV01@@Z 10002770 f i IexThrowErrnoExc.obj
 0001:000017b0       ??0EdomExc@Iex@@QAE@ABV01@@Z 100027b0 f i IexThrowErrnoExc.obj
 0001:000017f0       ??0ErangeExc@Iex@@QAE@ABV01@@Z 100027f0 f i IexThrowErrnoExc.obj
 0001:00001830       ??0EdeadlkExc@Iex@@QAE@ABV01@@Z 10002830 f i IexThrowErrnoExc.obj
 0001:00001870       ??0EnolckExc@Iex@@QAE@ABV01@@Z 10002870 f i IexThrowErrnoExc.obj
 0001:000018b0       ??0EnametoolongExc@Iex@@QAE@ABV01@@Z 100028b0 f i IexThrowErrnoExc.obj
 0001:000018f0       ??0EilseqExc@Iex@@QAE@ABV01@@Z 100028f0 f i IexThrowErrnoExc.obj
 0001:00001930       ??0EnosysExc@Iex@@QAE@ABV01@@Z 10002930 f i IexThrowErrnoExc.obj
 0001:00001970       ??0EnotemptyExc@Iex@@QAE@ABV01@@Z 10002970 f i IexThrowErrnoExc.obj
 0001:000019b0       ??0?$basic_string@DU?$char_traits@D@std@@V?$allocator@D@2@@std@@QAE@ABV01@@Z 100029b0 f   msvcprt:MSVCP80.dll
 0001:000019b6       ??0?$_String_val@DV?$allocator@D@std@@@std@@QAE@ABV01@@Z 100029b6 f   msvcprt:MSVCP80.dll
 0001:000019bc       __RTC_CheckEsp             100029bc f   MSVCRT:stack.obj
 0001:000019df       @_RTC_CheckStackVars@8     100029df f   MSVCRT:stack.obj
 0001:00001a39       ??_Etype_info@@UAEPAXI@Z   10002a39 f i MSVCRT:ti_inst.obj
 0001:00001a82       ??3@YAXPAX@Z               10002a82 f   MSVCRT:MSVCR80.dll
 0001:00001a88       ___CxxFrameHandler3        10002a88 f   MSVCRT:MSVCR80.dll
 0001:00001a8e       @__security_check_cookie@4 10002a8e f   MSVCRT:secchk.obj
 0001:00001a9e       __CxxThrowException@8      10002a9e f   MSVCRT:MSVCR80.dll
 0001:00001aa4       ??0exception@std@@QAE@ABV01@@Z 10002aa4 f   MSVCRT:MSVCR80.dll
 0001:00001af7       __CRT_INIT@12              10002af7 f   MSVCRT:crtdll.obj
 0001:00001dac       __DllMainCRTStartup@12     10002dac f   MSVCRT:crtdll.obj
 0001:00001dcd       ?_RTC_GetErrorFunc@@YAP6AHHPBDH00ZZPBX@Z 10002dcd f   MSVCRT:userapi.obj
 0001:00001dd3       ?_RTC_GetErrorFuncW@@YAP6AHHPB_WH00ZZPBX@Z 10002dd3 f   MSVCRT:userapi.obj
 0001:00002079       ?_RTC_Failure@@YAXPAXH@Z   10003079 f   MSVCRT:error.obj
 0001:000020b1       ?_RTC_StackFailure@@YAXPAXPBD@Z 100030b1 f   MSVCRT:error.obj
 0001:000021a2       ?__ArrayUnwind@@YGXPAXIHP6EX0@Z@Z 100031a2 f   MSVCRT:ehvecdtr.obj
 0001:00002200       ??_M@YGXPAXIHP6EX0@Z@Z     10003200 f   MSVCRT:ehvecdtr.obj
 0001:00002263       ___report_gsfailure        10003263 f   MSVCRT:gs_report.obj
 0001:00002367       ___clean_type_info_names   10003367 f   MSVCRT:tncleanup.obj
 0001:00002373       __onexit                   10003373 f   MSVCRT:atonexit.obj
 0001:00002412       _atexit                    10003412 f   MSVCRT:atonexit.obj
 0001:00002424       __RTC_Initialize           10003424 f   MSVCRT:initsect.obj
 0001:00002448       __RTC_Terminate            10003448 f   MSVCRT:initsect.obj
 0001:00002470       __ValidateImageBase        10003470 f   MSVCRT:pesect.obj
 0001:000024a0       __FindPESection            100034a0 f   MSVCRT:pesect.obj
 0001:000024e2       __IsNonwritableInCurrentImage 100034e2 f   MSVCRT:pesect.obj
 0001:0000254e       __initterm                 1000354e f   MSVCRT:MSVCR80.dll
 0001:00002554       __initterm_e               10003554 f   MSVCRT:MSVCR80.dll
 0001:0000255a       __amsg_exit                1000355a f   MSVCRT:MSVCR80.dll
 0001:00002560       ___CppXcptFilter           10003560 f   MSVCRT:MSVCR80.dll
 0001:00002566       _DllMain@12                10003566 f   MSVCRT:dllmain.obj
 0001:00002588       __SEH_prolog4              10003588 f   MSVCRT:sehprolg4.obj
 0001:000025cd       __SEH_epilog4              100035cd f   MSVCRT:sehprolg4.obj
 0001:000025e1       __except_handler4          100035e1 f   MSVCRT:chandler4gs.obj
 0001:00002604       ___security_init_cookie    10003604 f   MSVCRT:gs_support.obj
 0001:000027ef       ?_RTC_GetSrcLine@@YAHPAEPA_WKPAH1K@Z 100037ef f   MSVCRT:pdblkup.obj
 0001:00002a66       ?terminate@@YAXXZ          10003a66 f   MSVCRT:MSVCR80.dll
 0001:00002a6c       ?_type_info_dtor_internal_method@type_info@@QAEXXZ 10003a6c f   MSVCRT:MSVCR80.dll
 0001:00002a6c       ??1type_info@@UAE@XZ       10003a6c f   MSVCRT:MSVCR80.dll
 0001:00002a72       __crt_debugger_hook        10003a72 f   MSVCRT:MSVCR80.dll
 0001:00002a78       ___clean_type_info_names_internal 10003a78 f   MSVCRT:MSVCR80.dll
 0001:00002a7e       __unlock                   10003a7e f   MSVCRT:MSVCR80.dll
 0001:00002a84       ___dllonexit               10003a84 f   MSVCRT:MSVCR80.dll
 0001:00002a8a       __lock                     10003a8a f   MSVCRT:MSVCR80.dll
 0001:00002a90       __except_handler4_common   10003a90 f   MSVCRT:MSVCR80.dll
 0002:00000000       __imp__Sleep@4             10004000     kernel32:KERNEL32.dll
 0002:00000004       __imp__InterlockedCompareExchange@12 10004004     kernel32:KERNEL32.dll
 0002:00000008       __imp__RaiseException@16   10004008     kernel32:KERNEL32.dll
 0002:0000000c       __imp__DebugBreak@0        1000400c     kernel32:KERNEL32.dll
 0002:00000010       __imp__WideCharToMultiByte@32 10004010     kernel32:KERNEL32.dll
 0002:00000014       __imp__IsDebuggerPresent@0 10004014     kernel32:KERNEL32.dll
 0002:00000018       __imp__MultiByteToWideChar@24 10004018     kernel32:KERNEL32.dll
 0002:0000001c       __imp__GetProcAddress@8    1000401c     kernel32:KERNEL32.dll
 0002:00000020       __imp__LoadLibraryA@4      10004020     kernel32:KERNEL32.dll
 0002:00000024       __imp__VirtualQuery@12     10004024     kernel32:KERNEL32.dll
 0002:00000028       __imp__GetModuleFileNameW@12 10004028     kernel32:KERNEL32.dll
 0002:0000002c       __imp__GetProcessHeap@0    1000402c     kernel32:KERNEL32.dll
 0002:00000030       __imp__HeapAlloc@12        10004030     kernel32:KERNEL32.dll
 0002:00000034       __imp__HeapFree@12         10004034     kernel32:KERNEL32.dll
 0002:00000038       __imp__FreeLibrary@4       10004038     kernel32:KERNEL32.dll
 0002:0000003c       __imp__GetSystemTimeAsFileTime@4 1000403c     kernel32:KERNEL32.dll
 0002:00000040       __imp__GetCurrentProcessId@0 10004040     kernel32:KERNEL32.dll
 0002:00000044       __imp__GetCurrentThreadId@0 10004044     kernel32:KERNEL32.dll
 0002:00000048       __imp__GetTickCount@0      10004048     kernel32:KERNEL32.dll
 0002:0000004c       __imp__QueryPerformanceCounter@4 1000404c     kernel32:KERNEL32.dll
 0002:00000050       __imp__DisableThreadLibraryCalls@4 10004050     kernel32:KERNEL32.dll
 0002:00000054       __imp__SetUnhandledExceptionFilter@4 10004054     kernel32:KERNEL32.dll
 0002:00000058       __imp__UnhandledExceptionFilter@4 10004058     kernel32:KERNEL32.dll
 0002:0000005c       __imp__GetCurrentProcess@0 1000405c     kernel32:KERNEL32.dll
 0002:00000060       __imp__TerminateProcess@8  10004060     kernel32:KERNEL32.dll
 0002:00000064       __imp__InterlockedExchange@8 10004064     kernel32:KERNEL32.dll
 0002:00000068       \177KERNEL32_NULL_THUNK_DATA 10004068     kernel32:KERNEL32.dll
 0002:0000006c       __imp_??0?$_String_val@DV?$allocator@D@std@@@std@@QAE@ABV01@@Z 1000406c     msvcprt:MSVCP80.dll
 0002:00000070       __imp_?find@?$basic_string@DU?$char_traits@D@std@@V?$allocator@D@2@@std@@QBEIPBDI@Z 10004070     msvcprt:MSVCP80.dll
 0002:00000074       __imp_?replace@?$basic_string@DU?$char_traits@D@std@@V?$allocator@D@2@@std@@QAEAAV12@IIPBDI@Z 10004074     msvcprt:MSVCP80.dll
 0002:00000078       __imp_?append@?$basic_string@DU?$char_traits@D@std@@V?$allocator@D@2@@std@@QAEAAV12@ABV12@@Z 10004078     msvcprt:MSVCP80.dll
 0002:0000007c       __imp_?assign@?$basic_string@DU?$char_traits@D@std@@V?$allocator@D@2@@std@@QAEAAV12@ABV12@@Z 1000407c     msvcprt:MSVCP80.dll
 0002:00000080       __imp_?c_str@?$basic_string@DU?$char_traits@D@std@@V?$allocator@D@2@@std@@QBEPBDXZ 10004080     msvcprt:MSVCP80.dll
 0002:00000084       __imp_??1?$basic_string@DU?$char_traits@D@std@@V?$allocator@D@2@@std@@QAE@XZ 10004084     msvcprt:MSVCP80.dll
 0002:00000088       __imp_?str@?$basic_stringstream@DU?$char_traits@D@std@@V?$allocator@D@2@@std@@QBE?AV?$basic_string@DU?$char_traits@D@std@@V?$allocator@D@2@@2@XZ 10004088     msvcprt:MSVCP80.dll
 0002:0000008c       __imp_??0?$basic_string@DU?$char_traits@D@std@@V?$allocator@D@2@@std@@QAE@PBD@Z 1000408c     msvcprt:MSVCP80.dll
 0002:00000090       __imp_??0?$basic_string@DU?$char_traits@D@std@@V?$allocator@D@2@@std@@QAE@ABV01@@Z 10004090     msvcprt:MSVCP80.dll
 0002:00000094       \177MSVCP80_NULL_THUNK_DATA 10004094     msvcprt:MSVCP80.dll
 0002:00000098       __imp___except_handler4_common 10004098     MSVCRT:MSVCR80.dll
 0002:0000009c       __imp___onexit             1000409c     MSVCRT:MSVCR80.dll
 0002:000000a0       __imp___lock               100040a0     MSVCRT:MSVCR80.dll
 0002:000000a4       __imp____dllonexit         100040a4     MSVCRT:MSVCR80.dll
 0002:000000a8       __imp___unlock             100040a8     MSVCRT:MSVCR80.dll
 0002:000000ac       __imp___crt_debugger_hook  100040ac     MSVCRT:MSVCR80.dll
 0002:000000b0       __imp_?_type_info_dtor_internal_method@type_info@@QAEXXZ 100040b0     MSVCRT:MSVCR80.dll
 0002:000000b4       __imp_?terminate@@YAXXZ    100040b4     MSVCRT:MSVCR80.dll
 0002:000000b8       __imp____CppXcptFilter     100040b8     MSVCRT:MSVCR80.dll
 0002:000000bc       __imp___adjust_fdiv        100040bc     MSVCRT:MSVCR80.dll
 0002:000000c0       __imp___amsg_exit          100040c0     MSVCRT:MSVCR80.dll
 0002:000000c4       __imp___initterm_e         100040c4     MSVCRT:MSVCR80.dll
 0002:000000c8       __imp___initterm           100040c8     MSVCRT:MSVCR80.dll
 0002:000000cc       __imp___decode_pointer     100040cc     MSVCRT:MSVCR80.dll
 0002:000000d0       __imp__free                100040d0     MSVCRT:MSVCR80.dll
 0002:000000d4       __imp___encoded_null       100040d4     MSVCRT:MSVCR80.dll
 0002:000000d8       __imp___malloc_crt         100040d8     MSVCRT:MSVCR80.dll
 0002:000000dc       __imp___encode_pointer     100040dc     MSVCRT:MSVCR80.dll
 0002:000000e0       __imp___errno              100040e0     MSVCRT:MSVCR80.dll
 0002:000000e4       __imp_??0exception@std@@QAE@ABV01@@Z 100040e4     MSVCRT:MSVCR80.dll
 0002:000000e8       __imp___CxxThrowException@8 100040e8     MSVCRT:MSVCR80.dll
 0002:000000ec       __imp__strerror            100040ec     MSVCRT:MSVCR80.dll
 0002:000000f0       __imp____CxxFrameHandler3  100040f0     MSVCRT:MSVCR80.dll
 0002:000000f4       __imp_??1exception@std@@UAE@XZ 100040f4     MSVCRT:MSVCR80.dll
 0002:000000f8       __imp_??3@YAXPAX@Z         100040f8     MSVCRT:MSVCR80.dll
 0002:000000fc       __imp_??0exception@std@@QAE@XZ 100040fc     MSVCRT:MSVCR80.dll
 0002:00000100       __imp____clean_type_info_names_internal 10004100     MSVCRT:MSVCR80.dll
 0002:00000104       \177MSVCR80_NULL_THUNK_DATA 10004104     MSVCRT:MSVCR80.dll
 0002:00000108       ___xc_a                    10004108     MSVCRT:cinitexe.obj
 0002:0000010c       ___xc_z                    1000410c     MSVCRT:cinitexe.obj
 0002:00000110       ___xi_a                    10004110     MSVCRT:cinitexe.obj
 0002:00000118       ___xi_z                    10004118     MSVCRT:cinitexe.obj
 0002:00000138       ??_7BaseExc@Iex@@6B@       10004138     IexBaseExc.obj
 0002:00000158       ??_7ErrnoExc@Iex@@6B@      10004158     IexThrowErrnoExc.obj
 0002:00000164       ??_7EnotemptyExc@Iex@@6B@  10004164     IexThrowErrnoExc.obj
 0002:00000170       ??_7EnosysExc@Iex@@6B@     10004170     IexThrowErrnoExc.obj
 0002:0000017c       ??_7EilseqExc@Iex@@6B@     1000417c     IexThrowErrnoExc.obj
 0002:00000188       ??_7EnametoolongExc@Iex@@6B@ 10004188     IexThrowErrnoExc.obj
 0002:00000194       ??_7EnolckExc@Iex@@6B@     10004194     IexThrowErrnoExc.obj
 0002:000001a0       ??_7EdeadlkExc@Iex@@6B@    100041a0     IexThrowErrnoExc.obj
 0002:000001ac       ??_7ErangeExc@Iex@@6B@     100041ac     IexThrowErrnoExc.obj
 0002:000001b8       ??_7EdomExc@Iex@@6B@       100041b8     IexThrowErrnoExc.obj
 0002:000001c4       ??_7EpipeExc@Iex@@6B@      100041c4     IexThrowErrnoExc.obj
 0002:000001d0       ??_7EmlinkExc@Iex@@6B@     100041d0     IexThrowErrnoExc.obj
 0002:000001dc       ??_7ErofsExc@Iex@@6B@      100041dc     IexThrowErrnoExc.obj
 0002:000001e8       ??_7EspipeExc@Iex@@6B@     100041e8     IexThrowErrnoExc.obj
 0002:000001f4       ??_7EnospcExc@Iex@@6B@     100041f4     IexThrowErrnoExc.obj
 0002:00000200       ??_7EfbigExc@Iex@@6B@      10004200     IexThrowErrnoExc.obj
 0002:0000020c       ??_7EnottyExc@Iex@@6B@     1000420c     IexThrowErrnoExc.obj
 0002:00000218       ??_7EmfileExc@Iex@@6B@     10004218     IexThrowErrnoExc.obj
 0002:00000224       ??_7EnfileExc@Iex@@6B@     10004224     IexThrowErrnoExc.obj
 0002:00000230       ??_7EinvalExc@Iex@@6B@     10004230     IexThrowErrnoExc.obj
 0002:0000023c       ??_7EisdirExc@Iex@@6B@     1000423c     IexThrowErrnoExc.obj
 0002:00000248       ??_7EnotdirExc@Iex@@6B@    10004248     IexThrowErrnoExc.obj
 0002:00000254       ??_7EnodevExc@Iex@@6B@     10004254     IexThrowErrnoExc.obj
 0002:00000260       ??_7ExdevExc@Iex@@6B@      10004260     IexThrowErrnoExc.obj
 0002:0000026c       ??_7EexistExc@Iex@@6B@     1000426c     IexThrowErrnoExc.obj
 0002:00000278       ??_7EbusyExc@Iex@@6B@      10004278     IexThrowErrnoExc.obj
 0002:00000284       ??_7EfaultExc@Iex@@6B@     10004284     IexThrowErrnoExc.obj
 0002:00000290       ??_7EaccesExc@Iex@@6B@     10004290     IexThrowErrnoExc.obj
 0002:0000029c       ??_7EnomemExc@Iex@@6B@     1000429c     IexThrowErrnoExc.obj
 0002:000002a8       ??_7EagainExc@Iex@@6B@     100042a8     IexThrowErrnoExc.obj
 0002:000002b4       ??_7EchildExc@Iex@@6B@     100042b4     IexThrowErrnoExc.obj
 0002:000002c0       ??_7EbadfExc@Iex@@6B@      100042c0     IexThrowErrnoExc.obj
 0002:000002cc       ??_7EnoexecExc@Iex@@6B@    100042cc     IexThrowErrnoExc.obj
 0002:000002d8       ??_7E2bigExc@Iex@@6B@      100042d8     IexThrowErrnoExc.obj
 0002:000002e4       ??_7EnxioExc@Iex@@6B@      100042e4     IexThrowErrnoExc.obj
 0002:000002f0       ??_7EioExc@Iex@@6B@        100042f0     IexThrowErrnoExc.obj
 0002:000002fc       ??_7EintrExc@Iex@@6B@      100042fc     IexThrowErrnoExc.obj
 0002:00000308       ??_7EsrchExc@Iex@@6B@      10004308     IexThrowErrnoExc.obj
 0002:00000314       ??_7EnoentExc@Iex@@6B@     10004314     IexThrowErrnoExc.obj
 0002:00000320       ??_7EpermExc@Iex@@6B@      10004320     IexThrowErrnoExc.obj
 0002:0000032c       ??_7type_info@@6B@         1000432c     MSVCRT:ti_inst.obj
 0002:00000330       __pDefaultRawDllMain       10004330     MSVCRT:crtdll.obj
 0002:00000330       __pRawDllMain              10004330     MSVCRT:crtdll.obj
 0002:00000334       ??_C@_0BP@OGBCLIBO@Stack?5around?5_alloca?5corrupted?$AA@ 10004334     MSVCRT:userapi.obj
 0002:00000354       ??_C@_0CK@CNLNOEPB@Local?5variable?5used?5before?5initi@ 10004354     MSVCRT:userapi.obj
 0002:00000380       ??_C@_0BI@CIGMDCBH@Stack?5memory?5corruption?$AA@ 10004380     MSVCRT:userapi.obj
 0002:00000398       ??_C@_0CK@FEGOIOPB@Cast?5to?5smaller?5type?5causing?5los@ 10004398     MSVCRT:userapi.obj
 0002:000003c4       ??_C@_0BJ@HEGAHDFO@Stack?5pointer?5corruption?$AA@ 100043c4     MSVCRT:userapi.obj
 0002:000003e0       ??_C@_0BO@GNIAFIKK@Unknown?5Runtime?5Check?5Error?6?$AN?$AA@ 100043e0     MSVCRT:error.obj
 0002:00000400       ??_C@_0CM@NGINOKPC@Stack?5memory?5around?5_alloca?5was?5@ 10004400     MSVCRT:error.obj
 0002:0000042c       ??_C@_0DG@HKJMLLLP@A?5local?5variable?5was?5used?5before@ 1000442c     MSVCRT:error.obj
 0002:00000464       ??_C@_0BN@FFOINMNJ@Stack?5memory?5was?5corrupted?6?$AN?$AA@ 10004464     MSVCRT:error.obj
 0002:00000488       ??_C@_0BBN@GPMLNJCF@A?5cast?5to?5a?5smaller?5data?5type?5ha@ 10004488     MSVCRT:error.obj
 0002:000005a8       ??_C@_0NN@NGPKDKPD@The?5value?5of?5ESP?5was?5not?5properl@ 100045a8     MSVCRT:error.obj
 0002:00000708       ??_C@_0CA@IODNCDPG@Run?9Time?5Check?5Failure?5?$CD?$CFd?5?9?5?$CFs?$AA@ 10004708     MSVCRT:error.obj
 0002:00000728       ??_C@_0BE@GNBOBNCK@Unknown?5Module?5Name?$AA@ 10004728     MSVCRT:error.obj
 0002:0000073c       ??_C@_0BB@PFFGGCJP@Unknown?5Filename?$AA@ 1000473c     MSVCRT:error.obj
 0002:00000750       ??_C@_1EA@NFKNIFJP@?$AAR?$AAu?$AAn?$AA?9?$AAT?$AAi?$AAm?$AAe?$AA?5?$AAC?$AAh?$AAe?$AAc?$AAk?$AA?5?$AAF?$AAa?$AAi?$AAl?$AAu?$AAr?$AAe?$AA?5?$AA?$CD?$AA?$CF?$AAd?$AA?5?$AA?9?$AA?5?$AA?$CF?$AAs?$AA?$AA@ 10004750     MSVCRT:error.obj
 0002:00000790       ??_C@_1GM@OLMCBDMB@?$AAR?$AAu?$AAn?$AAt?$AAi?$AAm?$AAe?$AA?5?$AAC?$AAh?$AAe?$AAc?$AAk?$AA?5?$AAE?$AAr?$AAr?$AAo?$AAr?$AA?4?$AA?6?$AA?$AN?$AA?5?$AAU?$AAn?$AAa?$AAb?$AAl?$AAe?$AA?5?$AAt?$AAo@ 10004790     MSVCRT:error.obj
 0002:000007fc       ??_C@_0CG@IAFNJNEE@Stack?5corrupted?5near?5unknown?5var@ 100047fc     MSVCRT:error.obj
 0002:0000082c       ??_C@_0M@EKFFODEC@MSPDB80?4DLL?$AA@ 1000482c     MSVCRT:pdblkup.obj
 0002:00000838       ??_C@_0BF@BMIHBHCA@EnvironmentDirectory?$AA@ 10004838     MSVCRT:pdblkup.obj
 0002:00000850       ??_C@_0CN@EAEOKKOC@SOFTWARE?2Microsoft?2VisualStudio?2@ 10004850     MSVCRT:pdblkup.obj
 0002:00000880       ??_C@_0M@HLOHPNFA@RegCloseKey?$AA@ 10004880     MSVCRT:pdblkup.obj
 0002:0000088c       ??_C@_0BB@HHEIPGME@RegQueryValueExA?$AA@ 1000488c     MSVCRT:pdblkup.obj
 0002:000008a0       ??_C@_0O@DCOGKJGG@RegOpenKeyExA?$AA@ 100048a0     MSVCRT:pdblkup.obj
 0002:000008b0       ??_C@_0N@JJPEKNFO@ADVAPI32?4DLL?$AA@ 100048b0     MSVCRT:pdblkup.obj
 0002:000008c0       ??_C@_01KDCPPGHE@r?$AA@    100048c0     MSVCRT:pdblkup.obj
 0002:000008c4       ??_C@_0BB@KCIACLNC@PDBOpenValidate5?$AA@ 100048c4     MSVCRT:pdblkup.obj
 0002:000008d8       __load_config_used         100048d8     MSVCRT:loadcfg.obj
 0002:00000920       ??_R4BaseExc@Iex@@6B@      10004920     IexBaseExc.obj
 0002:00000934       ??_R3BaseExc@Iex@@8        10004934     IexBaseExc.obj
 0002:00000944       ??_R2BaseExc@Iex@@8        10004944     IexBaseExc.obj
 0002:00000960       ??_R1A@?0A@EA@BaseExc@Iex@@8 10004960     IexBaseExc.obj
 0002:0000097c       ??_R1M@?0A@EA@?$basic_string@DU?$char_traits@D@std@@V?$allocator@D@2@@std@@8 1000497c     IexBaseExc.obj
 0002:00000998       ??_R3?$basic_string@DU?$char_traits@D@std@@V?$allocator@D@2@@std@@8 10004998     IexBaseExc.obj
 0002:000009a8       ??_R2?$basic_string@DU?$char_traits@D@std@@V?$allocator@D@2@@std@@8 100049a8     IexBaseExc.obj
 0002:000009bc       ??_R1A@?0A@EA@?$basic_string@DU?$char_traits@D@std@@V?$allocator@D@2@@std@@8 100049bc     IexBaseExc.obj
 0002:000009d8       ??_R1A@?0A@EA@?$_String_val@DV?$allocator@D@std@@@std@@8 100049d8     IexBaseExc.obj
 0002:000009f4       ??_R3?$_String_val@DV?$allocator@D@std@@@std@@8 100049f4     IexBaseExc.obj
 0002:00000a04       ??_R2?$_String_val@DV?$allocator@D@std@@@std@@8 10004a04     IexBaseExc.obj
 0002:00000a14       ??_R1A@?0A@EA@_String_base@std@@8 10004a14     IexBaseExc.obj
 0002:00000a30       ??_R3_String_base@std@@8   10004a30     IexBaseExc.obj
 0002:00000a40       ??_R2_String_base@std@@8   10004a40     IexBaseExc.obj
 0002:00000a4c       ??_R1A@?0A@EA@_Container_base@std@@8 10004a4c     IexBaseExc.obj
 0002:00000a68       ??_R3_Container_base@std@@8 10004a68     IexBaseExc.obj
 0002:00000a78       ??_R2_Container_base@std@@8 10004a78     IexBaseExc.obj
 0002:00000a80       ??_R1M@?0A@EA@?$_String_val@DV?$allocator@D@std@@@std@@8 10004a80     IexBaseExc.obj
 0002:00000a9c       ??_R1M@?0A@EA@_String_base@std@@8 10004a9c     IexBaseExc.obj
 0002:00000ab8       ??_R1M@?0A@EA@_Container_base@std@@8 10004ab8     IexBaseExc.obj
 0002:00000ad4       ??_R1A@?0A@EA@exception@std@@8 10004ad4     IexBaseExc.obj
 0002:00000af0       ??_R3exception@std@@8      10004af0     IexBaseExc.obj
 0002:00000b00       ??_R2exception@std@@8      10004b00     IexBaseExc.obj
 0002:00000b08       ??_R4EpermExc@Iex@@6B@     10004b08     IexThrowErrnoExc.obj
 0002:00000b1c       ??_R3EpermExc@Iex@@8       10004b1c     IexThrowErrnoExc.obj
 0002:00000b2c       ??_R2EpermExc@Iex@@8       10004b2c     IexThrowErrnoExc.obj
 0002:00000b50       ??_R1A@?0A@EA@EpermExc@Iex@@8 10004b50     IexThrowErrnoExc.obj
 0002:00000b6c       ??_R1A@?0A@EA@ErrnoExc@Iex@@8 10004b6c     IexThrowErrnoExc.obj
 0002:00000b88       ??_R3ErrnoExc@Iex@@8       10004b88     IexThrowErrnoExc.obj
 0002:00000b98       ??_R2ErrnoExc@Iex@@8       10004b98     IexThrowErrnoExc.obj
 0002:00000bb8       ??_R4EnoentExc@Iex@@6B@    10004bb8     IexThrowErrnoExc.obj
 0002:00000bcc       ??_R3EnoentExc@Iex@@8      10004bcc     IexThrowErrnoExc.obj
 0002:00000bdc       ??_R2EnoentExc@Iex@@8      10004bdc     IexThrowErrnoExc.obj
 0002:00000c00       ??_R1A@?0A@EA@EnoentExc@Iex@@8 10004c00     IexThrowErrnoExc.obj
 0002:00000c1c       ??_R4EsrchExc@Iex@@6B@     10004c1c     IexThrowErrnoExc.obj
 0002:00000c30       ??_R3EsrchExc@Iex@@8       10004c30     IexThrowErrnoExc.obj
 0002:00000c40       ??_R2EsrchExc@Iex@@8       10004c40     IexThrowErrnoExc.obj
 0002:00000c64       ??_R1A@?0A@EA@EsrchExc@Iex@@8 10004c64     IexThrowErrnoExc.obj
 0002:00000c80       ??_R4EintrExc@Iex@@6B@     10004c80     IexThrowErrnoExc.obj
 0002:00000c94       ??_R3EintrExc@Iex@@8       10004c94     IexThrowErrnoExc.obj
 0002:00000ca4       ??_R2EintrExc@Iex@@8       10004ca4     IexThrowErrnoExc.obj
 0002:00000cc8       ??_R1A@?0A@EA@EintrExc@Iex@@8 10004cc8     IexThrowErrnoExc.obj
 0002:00000ce4       ??_R4EioExc@Iex@@6B@       10004ce4     IexThrowErrnoExc.obj
 0002:00000cf8       ??_R3EioExc@Iex@@8         10004cf8     IexThrowErrnoExc.obj
 0002:00000d08       ??_R2EioExc@Iex@@8         10004d08     IexThrowErrnoExc.obj
 0002:00000d2c       ??_R1A@?0A@EA@EioExc@Iex@@8 10004d2c     IexThrowErrnoExc.obj
 0002:00000d48       ??_R4EnxioExc@Iex@@6B@     10004d48     IexThrowErrnoExc.obj
 0002:00000d5c       ??_R3EnxioExc@Iex@@8       10004d5c     IexThrowErrnoExc.obj
 0002:00000d6c       ??_R2EnxioExc@Iex@@8       10004d6c     IexThrowErrnoExc.obj
 0002:00000d90       ??_R1A@?0A@EA@EnxioExc@Iex@@8 10004d90     IexThrowErrnoExc.obj
 0002:00000dac       ??_R4E2bigExc@Iex@@6B@     10004dac     IexThrowErrnoExc.obj
 0002:00000dc0       ??_R3E2bigExc@Iex@@8       10004dc0     IexThrowErrnoExc.obj
 0002:00000dd0       ??_R2E2bigExc@Iex@@8       10004dd0     IexThrowErrnoExc.obj
 0002:00000df4       ??_R1A@?0A@EA@E2bigExc@Iex@@8 10004df4     IexThrowErrnoExc.obj
 0002:00000e10       ??_R4EnoexecExc@Iex@@6B@   10004e10     IexThrowErrnoExc.obj
 0002:00000e24       ??_R3EnoexecExc@Iex@@8     10004e24     IexThrowErrnoExc.obj
 0002:00000e34       ??_R2EnoexecExc@Iex@@8     10004e34     IexThrowErrnoExc.obj
 0002:00000e58       ??_R1A@?0A@EA@EnoexecExc@Iex@@8 10004e58     IexThrowErrnoExc.obj
 0002:00000e74       ??_R4EbadfExc@Iex@@6B@     10004e74     IexThrowErrnoExc.obj
 0002:00000e88       ??_R3EbadfExc@Iex@@8       10004e88     IexThrowErrnoExc.obj
 0002:00000e98       ??_R2EbadfExc@Iex@@8       10004e98     IexThrowErrnoExc.obj
 0002:00000ebc       ??_R1A@?0A@EA@EbadfExc@Iex@@8 10004ebc     IexThrowErrnoExc.obj
 0002:00000ed8       ??_R4EchildExc@Iex@@6B@    10004ed8     IexThrowErrnoExc.obj
 0002:00000eec       ??_R3EchildExc@Iex@@8      10004eec     IexThrowErrnoExc.obj
 0002:00000efc       ??_R2EchildExc@Iex@@8      10004efc     IexThrowErrnoExc.obj
 0002:00000f20       ??_R1A@?0A@EA@EchildExc@Iex@@8 10004f20     IexThrowErrnoExc.obj
 0002:00000f3c       ??_R4EagainExc@Iex@@6B@    10004f3c     IexThrowErrnoExc.obj
 0002:00000f50       ??_R3EagainExc@Iex@@8      10004f50     IexThrowErrnoExc.obj
 0002:00000f60       ??_R2EagainExc@Iex@@8      10004f60     IexThrowErrnoExc.obj
 0002:00000f84       ??_R1A@?0A@EA@EagainExc@Iex@@8 10004f84     IexThrowErrnoExc.obj
 0002:00000fa0       ??_R4EnomemExc@Iex@@6B@    10004fa0     IexThrowErrnoExc.obj
 0002:00000fb4       ??_R3EnomemExc@Iex@@8      10004fb4     IexThrowErrnoExc.obj
 0002:00000fc4       ??_R2EnomemExc@Iex@@8      10004fc4     IexThrowErrnoExc.obj
 0002:00000fe8       ??_R1A@?0A@EA@EnomemExc@Iex@@8 10004fe8     IexThrowErrnoExc.obj
 0002:00001004       ??_R4EaccesExc@Iex@@6B@    10005004     IexThrowErrnoExc.obj
 0002:00001018       ??_R3EaccesExc@Iex@@8      10005018     IexThrowErrnoExc.obj
 0002:00001028       ??_R2EaccesExc@Iex@@8      10005028     IexThrowErrnoExc.obj
 0002:0000104c       ??_R1A@?0A@EA@EaccesExc@Iex@@8 1000504c     IexThrowErrnoExc.obj
 0002:00001068       ??_R4EfaultExc@Iex@@6B@    10005068     IexThrowErrnoExc.obj
 0002:0000107c       ??_R3EfaultExc@Iex@@8      1000507c     IexThrowErrnoExc.obj
 0002:0000108c       ??_R2EfaultExc@Iex@@8      1000508c     IexThrowErrnoExc.obj
 0002:000010b0       ??_R1A@?0A@EA@EfaultExc@Iex@@8 100050b0     IexThrowErrnoExc.obj
 0002:000010cc       ??_R4EbusyExc@Iex@@6B@     100050cc     IexThrowErrnoExc.obj
 0002:000010e0       ??_R3EbusyExc@Iex@@8       100050e0     IexThrowErrnoExc.obj
 0002:000010f0       ??_R2EbusyExc@Iex@@8       100050f0     IexThrowErrnoExc.obj
 0002:00001114       ??_R1A@?0A@EA@EbusyExc@Iex@@8 10005114     IexThrowErrnoExc.obj
 0002:00001130       ??_R4EexistExc@Iex@@6B@    10005130     IexThrowErrnoExc.obj
 0002:00001144       ??_R3EexistExc@Iex@@8      10005144     IexThrowErrnoExc.obj
 0002:00001154       ??_R2EexistExc@Iex@@8      10005154     IexThrowErrnoExc.obj
 0002:00001178       ??_R1A@?0A@EA@EexistExc@Iex@@8 10005178     IexThrowErrnoExc.obj
 0002:00001194       ??_R4ExdevExc@Iex@@6B@     10005194     IexThrowErrnoExc.obj
 0002:000011a8       ??_R3ExdevExc@Iex@@8       100051a8     IexThrowErrnoExc.obj
 0002:000011b8       ??_R2ExdevExc@Iex@@8       100051b8     IexThrowErrnoExc.obj
 0002:000011dc       ??_R1A@?0A@EA@ExdevExc@Iex@@8 100051dc     IexThrowErrnoExc.obj
 0002:000011f8       ??_R4EnodevExc@Iex@@6B@    100051f8     IexThrowErrnoExc.obj
 0002:0000120c       ??_R3EnodevExc@Iex@@8      1000520c     IexThrowErrnoExc.obj
 0002:0000121c       ??_R2EnodevExc@Iex@@8      1000521c     IexThrowErrnoExc.obj
 0002:00001240       ??_R1A@?0A@EA@EnodevExc@Iex@@8 10005240     IexThrowErrnoExc.obj
 0002:0000125c       ??_R4EnotdirExc@Iex@@6B@   1000525c     IexThrowErrnoExc.obj
 0002:00001270       ??_R3EnotdirExc@Iex@@8     10005270     IexThrowErrnoExc.obj
 0002:00001280       ??_R2EnotdirExc@Iex@@8     10005280     IexThrowErrnoExc.obj
 0002:000012a4       ??_R1A@?0A@EA@EnotdirExc@Iex@@8 100052a4     IexThrowErrnoExc.obj
 0002:000012c0       ??_R4EisdirExc@Iex@@6B@    100052c0     IexThrowErrnoExc.obj
 0002:000012d4       ??_R3EisdirExc@Iex@@8      100052d4     IexThrowErrnoExc.obj
 0002:000012e4       ??_R2EisdirExc@Iex@@8      100052e4     IexThrowErrnoExc.obj
 0002:00001308       ??_R1A@?0A@EA@EisdirExc@Iex@@8 10005308     IexThrowErrnoExc.obj
 0002:00001324       ??_R4EinvalExc@Iex@@6B@    10005324     IexThrowErrnoExc.obj
 0002:00001338       ??_R3EinvalExc@Iex@@8      10005338     IexThrowErrnoExc.obj
 0002:00001348       ??_R2EinvalExc@Iex@@8      10005348     IexThrowErrnoExc.obj
 0002:0000136c       ??_R1A@?0A@EA@EinvalExc@Iex@@8 1000536c     IexThrowErrnoExc.obj
 0002:00001388       ??_R4EnfileExc@Iex@@6B@    10005388     IexThrowErrnoExc.obj
 0002:0000139c       ??_R3EnfileExc@Iex@@8      1000539c     IexThrowErrnoExc.obj
 0002:000013ac       ??_R2EnfileExc@Iex@@8      100053ac     IexThrowErrnoExc.obj
 0002:000013d0       ??_R1A@?0A@EA@EnfileExc@Iex@@8 100053d0     IexThrowErrnoExc.obj
 0002:000013ec       ??_R4EmfileExc@Iex@@6B@    100053ec     IexThrowErrnoExc.obj
 0002:00001400       ??_R3EmfileExc@Iex@@8      10005400     IexThrowErrnoExc.obj
 0002:00001410       ??_R2EmfileExc@Iex@@8      10005410     IexThrowErrnoExc.obj
 0002:00001434       ??_R1A@?0A@EA@EmfileExc@Iex@@8 10005434     IexThrowErrnoExc.obj
 0002:00001450       ??_R4EnottyExc@Iex@@6B@    10005450     IexThrowErrnoExc.obj
 0002:00001464       ??_R3EnottyExc@Iex@@8      10005464     IexThrowErrnoExc.obj
 0002:00001474       ??_R2EnottyExc@Iex@@8      10005474     IexThrowErrnoExc.obj
 0002:00001498       ??_R1A@?0A@EA@EnottyExc@Iex@@8 10005498     IexThrowErrnoExc.obj
 0002:000014b4       ??_R4EfbigExc@Iex@@6B@     100054b4     IexThrowErrnoExc.obj
 0002:000014c8       ??_R3EfbigExc@Iex@@8       100054c8     IexThrowErrnoExc.obj
 0002:000014d8       ??_R2EfbigExc@Iex@@8       100054d8     IexThrowErrnoExc.obj
 0002:000014fc       ??_R1A@?0A@EA@EfbigExc@Iex@@8 100054fc     IexThrowErrnoExc.obj
 0002:00001518       ??_R4EnospcExc@Iex@@6B@    10005518     IexThrowErrnoExc.obj
 0002:0000152c       ??_R3EnospcExc@Iex@@8      1000552c     IexThrowErrnoExc.obj
 0002:0000153c       ??_R2EnospcExc@Iex@@8      1000553c     IexThrowErrnoExc.obj
 0002:00001560       ??_R1A@?0A@EA@EnospcExc@Iex@@8 10005560     IexThrowErrnoExc.obj
 0002:0000157c       ??_R4EspipeExc@Iex@@6B@    1000557c     IexThrowErrnoExc.obj
 0002:00001590       ??_R3EspipeExc@Iex@@8      10005590     IexThrowErrnoExc.obj
 0002:000015a0       ??_R2EspipeExc@Iex@@8      100055a0     IexThrowErrnoExc.obj
 0002:000015c4       ??_R1A@?0A@EA@EspipeExc@Iex@@8 100055c4     IexThrowErrnoExc.obj
 0002:000015e0       ??_R4ErofsExc@Iex@@6B@     100055e0     IexThrowErrnoExc.obj
 0002:000015f4       ??_R3ErofsExc@Iex@@8       100055f4     IexThrowErrnoExc.obj
 0002:00001604       ??_R2ErofsExc@Iex@@8       10005604     IexThrowErrnoExc.obj
 0002:00001628       ??_R1A@?0A@EA@ErofsExc@Iex@@8 10005628     IexThrowErrnoExc.obj
 0002:00001644       ??_R4EmlinkExc@Iex@@6B@    10005644     IexThrowErrnoExc.obj
 0002:00001658       ??_R3EmlinkExc@Iex@@8      10005658     IexThrowErrnoExc.obj
 0002:00001668       ??_R2EmlinkExc@Iex@@8      10005668     IexThrowErrnoExc.obj
 0002:0000168c       ??_R1A@?0A@EA@EmlinkExc@Iex@@8 1000568c     IexThrowErrnoExc.obj
 0002:000016a8       ??_R4EpipeExc@Iex@@6B@     100056a8     IexThrowErrnoExc.obj
 0002:000016bc       ??_R3EpipeExc@Iex@@8       100056bc     IexThrowErrnoExc.obj
 0002:000016cc       ??_R2EpipeExc@Iex@@8       100056cc     IexThrowErrnoExc.obj
 0002:000016f0       ??_R1A@?0A@EA@EpipeExc@Iex@@8 100056f0     IexThrowErrnoExc.obj
 0002:0000170c       ??_R4EdomExc@Iex@@6B@      1000570c     IexThrowErrnoExc.obj
 0002:00001720       ??_R3EdomExc@Iex@@8        10005720     IexThrowErrnoExc.obj
 0002:00001730       ??_R2EdomExc@Iex@@8        10005730     IexThrowErrnoExc.obj
 0002:00001754       ??_R1A@?0A@EA@EdomExc@Iex@@8 10005754     IexThrowErrnoExc.obj
 0002:00001770       ??_R4ErangeExc@Iex@@6B@    10005770     IexThrowErrnoExc.obj
 0002:00001784       ??_R3ErangeExc@Iex@@8      10005784     IexThrowErrnoExc.obj
 0002:00001794       ??_R2ErangeExc@Iex@@8      10005794     IexThrowErrnoExc.obj
 0002:000017b8       ??_R1A@?0A@EA@ErangeExc@Iex@@8 100057b8     IexThrowErrnoExc.obj
 0002:000017d4       ??_R4EdeadlkExc@Iex@@6B@   100057d4     IexThrowErrnoExc.obj
 0002:000017e8       ??_R3EdeadlkExc@Iex@@8     100057e8     IexThrowErrnoExc.obj
 0002:000017f8       ??_R2EdeadlkExc@Iex@@8     100057f8     IexThrowErrnoExc.obj
 0002:0000181c       ??_R1A@?0A@EA@EdeadlkExc@Iex@@8 1000581c     IexThrowErrnoExc.obj
 0002:00001838       ??_R4EnolckExc@Iex@@6B@    10005838     IexThrowErrnoExc.obj
 0002:0000184c       ??_R3EnolckExc@Iex@@8      1000584c     IexThrowErrnoExc.obj
 0002:0000185c       ??_R2EnolckExc@Iex@@8      1000585c     IexThrowErrnoExc.obj
 0002:00001880       ??_R1A@?0A@EA@EnolckExc@Iex@@8 10005880     IexThrowErrnoExc.obj
 0002:0000189c       ??_R4EnametoolongExc@Iex@@6B@ 1000589c     IexThrowErrnoExc.obj
 0002:000018b0       ??_R3EnametoolongExc@Iex@@8 100058b0     IexThrowErrnoExc.obj
 0002:000018c0       ??_R2EnametoolongExc@Iex@@8 100058c0     IexThrowErrnoExc.obj
 0002:000018e4       ??_R1A@?0A@EA@EnametoolongExc@Iex@@8 100058e4     IexThrowErrnoExc.obj
 0002:00001900       ??_R4EilseqExc@Iex@@6B@    10005900     IexThrowErrnoExc.obj
 0002:00001914       ??_R3EilseqExc@Iex@@8      10005914     IexThrowErrnoExc.obj
 0002:00001924       ??_R2EilseqExc@Iex@@8      10005924     IexThrowErrnoExc.obj
 0002:00001948       ??_R1A@?0A@EA@EilseqExc@Iex@@8 10005948     IexThrowErrnoExc.obj
 0002:00001964       ??_R4EnosysExc@Iex@@6B@    10005964     IexThrowErrnoExc.obj
 0002:00001978       ??_R3EnosysExc@Iex@@8      10005978     IexThrowErrnoExc.obj
 0002:00001988       ??_R2EnosysExc@Iex@@8      10005988     IexThrowErrnoExc.obj
 0002:000019ac       ??_R1A@?0A@EA@EnosysExc@Iex@@8 100059ac     IexThrowErrnoExc.obj
 0002:000019c8       ??_R4EnotemptyExc@Iex@@6B@ 100059c8     IexThrowErrnoExc.obj
 0002:000019dc       ??_R3EnotemptyExc@Iex@@8   100059dc     IexThrowErrnoExc.obj
 0002:000019ec       ??_R2EnotemptyExc@Iex@@8   100059ec     IexThrowErrnoExc.obj
 0002:00001a10       ??_R1A@?0A@EA@EnotemptyExc@Iex@@8 10005a10     IexThrowErrnoExc.obj
 0002:00001a2c       ??_R4ErrnoExc@Iex@@6B@     10005a2c     IexThrowErrnoExc.obj
 0002:00001a40       ??_R4type_info@@6B@        10005a40     MSVCRT:ti_inst.obj
 0002:00001a54       ??_R3type_info@@8          10005a54     MSVCRT:ti_inst.obj
 0002:00001a64       ??_R2type_info@@8          10005a64     MSVCRT:ti_inst.obj
 0002:00001a6c       ??_R1A@?0A@EA@type_info@@8 10005a6c     MSVCRT:ti_inst.obj
 0002:00001a90       ___safe_se_handler_table   10005a90     <linker-defined>
 0002:00001aa0       ___rtc_iaa                 10005aa0     MSVCRT:initsect.obj
 0002:00001aa4       ___rtc_izz                 10005aa4     MSVCRT:initsect.obj
 0002:00001aa8       ___rtc_taa                 10005aa8     MSVCRT:initsect.obj
 0002:00001aac       ___rtc_tzz                 10005aac     MSVCRT:initsect.obj
 0002:00001b08       __TI7?AVErrnoExc@Iex@@     10005b08     IexThrowErrnoExc.obj
 0002:00001b18       __TI8?AVEnotemptyExc@Iex@@ 10005b18     IexThrowErrnoExc.obj
 0002:00001b28       __TI8?AVEnosysExc@Iex@@    10005b28     IexThrowErrnoExc.obj
 0002:00001b38       __TI8?AVEilseqExc@Iex@@    10005b38     IexThrowErrnoExc.obj
 0002:00001b48       __TI8?AVEnametoolongExc@Iex@@ 10005b48     IexThrowErrnoExc.obj
 0002:00001b58       __TI8?AVEnolckExc@Iex@@    10005b58     IexThrowErrnoExc.obj
 0002:00001b68       __TI8?AVEdeadlkExc@Iex@@   10005b68     IexThrowErrnoExc.obj
 0002:00001b78       __TI8?AVErangeExc@Iex@@    10005b78     IexThrowErrnoExc.obj
 0002:00001b88       __TI8?AVEdomExc@Iex@@      10005b88     IexThrowErrnoExc.obj
 0002:00001b98       __TI8?AVEpipeExc@Iex@@     10005b98     IexThrowErrnoExc.obj
 0002:00001ba8       __TI8?AVEmlinkExc@Iex@@    10005ba8     IexThrowErrnoExc.obj
 0002:00001bb8       __TI8?AVErofsExc@Iex@@     10005bb8     IexThrowErrnoExc.obj
 0002:00001bc8       __TI8?AVEspipeExc@Iex@@    10005bc8     IexThrowErrnoExc.obj
 0002:00001bd8       __TI8?AVEnospcExc@Iex@@    10005bd8     IexThrowErrnoExc.obj
 0002:00001be8       __TI8?AVEfbigExc@Iex@@     10005be8     IexThrowErrnoExc.obj
 0002:00001bf8       __TI8?AVEnottyExc@Iex@@    10005bf8     IexThrowErrnoExc.obj
 0002:00001c08       __TI8?AVEmfileExc@Iex@@    10005c08     IexThrowErrnoExc.obj
 0002:00001c18       __TI8?AVEnfileExc@Iex@@    10005c18     IexThrowErrnoExc.obj
 0002:00001c28       __TI8?AVEinvalExc@Iex@@    10005c28     IexThrowErrnoExc.obj
 0002:00001c38       __TI8?AVEisdirExc@Iex@@    10005c38     IexThrowErrnoExc.obj
 0002:00001c48       __TI8?AVEnotdirExc@Iex@@   10005c48     IexThrowErrnoExc.obj
 0002:00001c58       __TI8?AVEnodevExc@Iex@@    10005c58     IexThrowErrnoExc.obj
 0002:00001c68       __TI8?AVExdevExc@Iex@@     10005c68     IexThrowErrnoExc.obj
 0002:00001c78       __TI8?AVEexistExc@Iex@@    10005c78     IexThrowErrnoExc.obj
 0002:00001c88       __TI8?AVEbusyExc@Iex@@     10005c88     IexThrowErrnoExc.obj
 0002:00001c98       __TI8?AVEfaultExc@Iex@@    10005c98     IexThrowErrnoExc.obj
 0002:00001ca8       __TI8?AVEaccesExc@Iex@@    10005ca8     IexThrowErrnoExc.obj
 0002:00001cb8       __TI8?AVEnomemExc@Iex@@    10005cb8     IexThrowErrnoExc.obj
 0002:00001cc8       __TI8?AVEagainExc@Iex@@    10005cc8     IexThrowErrnoExc.obj
 0002:00001cd8       __TI8?AVEchildExc@Iex@@    10005cd8     IexThrowErrnoExc.obj
 0002:00001ce8       __TI8?AVEbadfExc@Iex@@     10005ce8     IexThrowErrnoExc.obj
 0002:00001cf8       __TI8?AVEnoexecExc@Iex@@   10005cf8     IexThrowErrnoExc.obj
 0002:00001d08       __TI8?AVE2bigExc@Iex@@     10005d08     IexThrowErrnoExc.obj
 0002:00001d18       __TI8?AVEnxioExc@Iex@@     10005d18     IexThrowErrnoExc.obj
 0002:00001d28       __TI8?AVEioExc@Iex@@       10005d28     IexThrowErrnoExc.obj
 0002:00001d38       __TI8?AVEintrExc@Iex@@     10005d38     IexThrowErrnoExc.obj
 0002:00001d48       __TI8?AVEsrchExc@Iex@@     10005d48     IexThrowErrnoExc.obj
 0002:00001d58       __TI8?AVEnoentExc@Iex@@    10005d58     IexThrowErrnoExc.obj
 0002:00001d68       __TI8?AVEpermExc@Iex@@     10005d68     IexThrowErrnoExc.obj
 0002:00001da4       __CTA8?AVEpermExc@Iex@@    10005da4     IexThrowErrnoExc.obj
 0002:00001dc8       __CT??_R0?AVEpermExc@Iex@@@8??0EpermExc@Iex@@QAE@ABV01@@Z68 10005dc8     IexThrowErrnoExc.obj
 0002:00001de4       __CT??_R0?AVErrnoExc@Iex@@@8??0ErrnoExc@Iex@@QAE@ABV01@@Z68 10005de4     IexThrowErrnoExc.obj
 0002:00001e00       __CT??_R0?AVBaseExc@Iex@@@8??0BaseExc@Iex@@QAE@ABV01@@Z68 10005e00     IexThrowErrnoExc.obj
 0002:00001e1c       __CT??_R0?AV?$basic_string@DU?$char_traits@D@std@@V?$allocator@D@2@@std@@@8??0?$basic_string@DU?$char_traits@D@std@@V?$allocator@D@2@@std@@QAE@ABV01@@Z2812 10005e1c     IexThrowErrnoExc.obj
 0002:00001e38       __CT??_R0?AV?$_String_val@DV?$allocator@D@std@@@std@@@8??0?$_String_val@DV?$allocator@D@std@@@std@@QAE@ABV01@@Z112 10005e38     IexThrowErrnoExc.obj
 0002:00001e54       __CT??_R0?AV_String_base@std@@@8112 10005e54     IexThrowErrnoExc.obj
 0002:00001e70       __CT??_R0?AU_Container_base@std@@@8112 10005e70     IexThrowErrnoExc.obj
 0002:00001e8c       __CT??_R0?AVexception@std@@@8??0exception@std@@QAE@ABV01@@Z12 10005e8c     IexThrowErrnoExc.obj
 0002:00001ea8       __CTA8?AVEnoentExc@Iex@@   10005ea8     IexThrowErrnoExc.obj
 0002:00001ecc       __CT??_R0?AVEnoentExc@Iex@@@8??0EnoentExc@Iex@@QAE@ABV01@@Z68 10005ecc     IexThrowErrnoExc.obj
 0002:00001ee8       __CTA8?AVEsrchExc@Iex@@    10005ee8     IexThrowErrnoExc.obj
 0002:00001f0c       __CT??_R0?AVEsrchExc@Iex@@@8??0EsrchExc@Iex@@QAE@ABV01@@Z68 10005f0c     IexThrowErrnoExc.obj
 0002:00001f28       __CTA8?AVEintrExc@Iex@@    10005f28     IexThrowErrnoExc.obj
 0002:00001f4c       __CT??_R0?AVEintrExc@Iex@@@8??0EintrExc@Iex@@QAE@ABV01@@Z68 10005f4c     IexThrowErrnoExc.obj
 0002:00001f68       __CTA8?AVEioExc@Iex@@      10005f68     IexThrowErrnoExc.obj
 0002:00001f8c       __CT??_R0?AVEioExc@Iex@@@8??0EioExc@Iex@@QAE@ABV01@@Z68 10005f8c     IexThrowErrnoExc.obj
 0002:00001fa8       __CTA8?AVEnxioExc@Iex@@    10005fa8     IexThrowErrnoExc.obj
 0002:00001fcc       __CT??_R0?AVEnxioExc@Iex@@@8??0EnxioExc@Iex@@QAE@ABV01@@Z68 10005fcc     IexThrowErrnoExc.obj
 0002:00001fe8       __CTA8?AVE2bigExc@Iex@@    10005fe8     IexThrowErrnoExc.obj
 0002:0000200c       __CT??_R0?AVE2bigExc@Iex@@@8??0E2bigExc@Iex@@QAE@ABV01@@Z68 1000600c     IexThrowErrnoExc.obj
 0002:00002028       __CTA8?AVEnoexecExc@Iex@@  10006028     IexThrowErrnoExc.obj
 0002:0000204c       __CT??_R0?AVEnoexecExc@Iex@@@8??0EnoexecExc@Iex@@QAE@ABV01@@Z68 1000604c     IexThrowErrnoExc.obj
 0002:00002068       __CTA8?AVEbadfExc@Iex@@    10006068     IexThrowErrnoExc.obj
 0002:0000208c       __CT??_R0?AVEbadfExc@Iex@@@8??0EbadfExc@Iex@@QAE@ABV01@@Z68 1000608c     IexThrowErrnoExc.obj
 0002:000020a8       __CTA8?AVEchildExc@Iex@@   100060a8     IexThrowErrnoExc.obj
 0002:000020cc       __CT??_R0?AVEchildExc@Iex@@@8??0EchildExc@Iex@@QAE@ABV01@@Z68 100060cc     IexThrowErrnoExc.obj
 0002:000020e8       __CTA8?AVEagainExc@Iex@@   100060e8     IexThrowErrnoExc.obj
 0002:0000210c       __CT??_R0?AVEagainExc@Iex@@@8??0EagainExc@Iex@@QAE@ABV01@@Z68 1000610c     IexThrowErrnoExc.obj
 0002:00002128       __CTA8?AVEnomemExc@Iex@@   10006128     IexThrowErrnoExc.obj
 0002:0000214c       __CT??_R0?AVEnomemExc@Iex@@@8??0EnomemExc@Iex@@QAE@ABV01@@Z68 1000614c     IexThrowErrnoExc.obj
 0002:00002168       __CTA8?AVEaccesExc@Iex@@   10006168     IexThrowErrnoExc.obj
 0002:0000218c       __CT??_R0?AVEaccesExc@Iex@@@8??0EaccesExc@Iex@@QAE@ABV01@@Z68 1000618c     IexThrowErrnoExc.obj
 0002:000021a8       __CTA8?AVEfaultExc@Iex@@   100061a8     IexThrowErrnoExc.obj
 0002:000021cc       __CT??_R0?AVEfaultExc@Iex@@@8??0EfaultExc@Iex@@QAE@ABV01@@Z68 100061cc     IexThrowErrnoExc.obj
 0002:000021e8       __CTA8?AVEbusyExc@Iex@@    100061e8     IexThrowErrnoExc.obj
 0002:0000220c       __CT??_R0?AVEbusyExc@Iex@@@8??0EbusyExc@Iex@@QAE@ABV01@@Z68 1000620c     IexThrowErrnoExc.obj
 0002:00002228       __CTA8?AVEexistExc@Iex@@   10006228     IexThrowErrnoExc.obj
 0002:0000224c       __CT??_R0?AVEexistExc@Iex@@@8??0EexistExc@Iex@@QAE@ABV01@@Z68 1000624c     IexThrowErrnoExc.obj
 0002:00002268       __CTA8?AVExdevExc@Iex@@    10006268     IexThrowErrnoExc.obj
 0002:0000228c       __CT??_R0?AVExdevExc@Iex@@@8??0ExdevExc@Iex@@QAE@ABV01@@Z68 1000628c     IexThrowErrnoExc.obj
 0002:000022a8       __CTA8?AVEnodevExc@Iex@@   100062a8     IexThrowErrnoExc.obj
 0002:000022cc       __CT??_R0?AVEnodevExc@Iex@@@8??0EnodevExc@Iex@@QAE@ABV01@@Z68 100062cc     IexThrowErrnoExc.obj
 0002:000022e8       __CTA8?AVEnotdirExc@Iex@@  100062e8     IexThrowErrnoExc.obj
 0002:0000230c       __CT??_R0?AVEnotdirExc@Iex@@@8??0EnotdirExc@Iex@@QAE@ABV01@@Z68 1000630c     IexThrowErrnoExc.obj
 0002:00002328       __CTA8?AVEisdirExc@Iex@@   10006328     IexThrowErrnoExc.obj
 0002:0000234c       __CT??_R0?AVEisdirExc@Iex@@@8??0EisdirExc@Iex@@QAE@ABV01@@Z68 1000634c     IexThrowErrnoExc.obj
 0002:00002368       __CTA8?AVEinvalExc@Iex@@   10006368     IexThrowErrnoExc.obj
 0002:0000238c       __CT??_R0?AVEinvalExc@Iex@@@8??0EinvalExc@Iex@@QAE@ABV01@@Z68 1000638c     IexThrowErrnoExc.obj
 0002:000023a8       __CTA8?AVEnfileExc@Iex@@   100063a8     IexThrowErrnoExc.obj
 0002:000023cc       __CT??_R0?AVEnfileExc@Iex@@@8??0EnfileExc@Iex@@QAE@ABV01@@Z68 100063cc     IexThrowErrnoExc.obj
 0002:000023e8       __CTA8?AVEmfileExc@Iex@@   100063e8     IexThrowErrnoExc.obj
 0002:0000240c       __CT??_R0?AVEmfileExc@Iex@@@8??0EmfileExc@Iex@@QAE@ABV01@@Z68 1000640c     IexThrowErrnoExc.obj
 0002:00002428       __CTA8?AVEnottyExc@Iex@@   10006428     IexThrowErrnoExc.obj
 0002:0000244c       __CT??_R0?AVEnottyExc@Iex@@@8??0EnottyExc@Iex@@QAE@ABV01@@Z68 1000644c     IexThrowErrnoExc.obj
 0002:00002468       __CTA8?AVEfbigExc@Iex@@    10006468     IexThrowErrnoExc.obj
 0002:0000248c       __CT??_R0?AVEfbigExc@Iex@@@8??0EfbigExc@Iex@@QAE@ABV01@@Z68 1000648c     IexThrowErrnoExc.obj
 0002:000024a8       __CTA8?AVEnospcExc@Iex@@   100064a8     IexThrowErrnoExc.obj
 0002:000024cc       __CT??_R0?AVEnospcExc@Iex@@@8??0EnospcExc@Iex@@QAE@ABV01@@Z68 100064cc     IexThrowErrnoExc.obj
 0002:000024e8       __CTA8?AVEspipeExc@Iex@@   100064e8     IexThrowErrnoExc.obj
 0002:0000250c       __CT??_R0?AVEspipeExc@Iex@@@8??0EspipeExc@Iex@@QAE@ABV01@@Z68 1000650c     IexThrowErrnoExc.obj
 0002:00002528       __CTA8?AVErofsExc@Iex@@    10006528     IexThrowErrnoExc.obj
 0002:0000254c       __CT??_R0?AVErofsExc@Iex@@@8??0ErofsExc@Iex@@QAE@ABV01@@Z68 1000654c     IexThrowErrnoExc.obj
 0002:00002568       __CTA8?AVEmlinkExc@Iex@@   10006568     IexThrowErrnoExc.obj
 0002:0000258c       __CT??_R0?AVEmlinkExc@Iex@@@8??0EmlinkExc@Iex@@QAE@ABV01@@Z68 1000658c     IexThrowErrnoExc.obj
 0002:000025a8       __CTA8?AVEpipeExc@Iex@@    100065a8     IexThrowErrnoExc.obj
 0002:000025cc       __CT??_R0?AVEpipeExc@Iex@@@8??0EpipeExc@Iex@@QAE@ABV01@@Z68 100065cc     IexThrowErrnoExc.obj
 0002:000025e8       __CTA8?AVEdomExc@Iex@@     100065e8     IexThrowErrnoExc.obj
 0002:0000260c       __CT??_R0?AVEdomExc@Iex@@@8??0EdomExc@Iex@@QAE@ABV01@@Z68 1000660c     IexThrowErrnoExc.obj
 0002:00002628       __CTA8?AVErangeExc@Iex@@   10006628     IexThrowErrnoExc.obj
 0002:0000264c       __CT??_R0?AVErangeExc@Iex@@@8??0ErangeExc@Iex@@QAE@ABV01@@Z68 1000664c     IexThrowErrnoExc.obj
 0002:00002668       __CTA8?AVEdeadlkExc@Iex@@  10006668     IexThrowErrnoExc.obj
 0002:0000268c       __CT??_R0?AVEdeadlkExc@Iex@@@8??0EdeadlkExc@Iex@@QAE@ABV01@@Z68 1000668c     IexThrowErrnoExc.obj
 0002:000026a8       __CTA8?AVEnolckExc@Iex@@   100066a8     IexThrowErrnoExc.obj
 0002:000026cc       __CT??_R0?AVEnolckExc@Iex@@@8??0EnolckExc@Iex@@QAE@ABV01@@Z68 100066cc     IexThrowErrnoExc.obj
 0002:000026e8       __CTA8?AVEnametoolongExc@Iex@@ 100066e8     IexThrowErrnoExc.obj
 0002:0000270c       __CT??_R0?AVEnametoolongExc@Iex@@@8??0EnametoolongExc@Iex@@QAE@ABV01@@Z68 1000670c     IexThrowErrnoExc.obj
 0002:00002728       __CTA8?AVEilseqExc@Iex@@   10006728     IexThrowErrnoExc.obj
 0002:0000274c       __CT??_R0?AVEilseqExc@Iex@@@8??0EilseqExc@Iex@@QAE@ABV01@@Z68 1000674c     IexThrowErrnoExc.obj
 0002:00002768       __CTA8?AVEnosysExc@Iex@@   10006768     IexThrowErrnoExc.obj
 0002:0000278c       __CT??_R0?AVEnosysExc@Iex@@@8??0EnosysExc@Iex@@QAE@ABV01@@Z68 1000678c     IexThrowErrnoExc.obj
 0002:000027a8       __CTA8?AVEnotemptyExc@Iex@@ 100067a8     IexThrowErrnoExc.obj
 0002:000027cc       __CT??_R0?AVEnotemptyExc@Iex@@@8??0EnotemptyExc@Iex@@QAE@ABV01@@Z68 100067cc     IexThrowErrnoExc.obj
 0002:000027e8       __CTA7?AVErrnoExc@Iex@@    100067e8     IexThrowErrnoExc.obj
 0002:000028ec       __IMPORT_DESCRIPTOR_MSVCP80 100068ec     msvcprt:MSVCP80.dll
 0002:00002900       __IMPORT_DESCRIPTOR_MSVCR80 10006900     MSVCRT:MSVCR80.dll
 0002:00002914       __IMPORT_DESCRIPTOR_KERNEL32 10006914     kernel32:KERNEL32.dll
 0002:00002928       __NULL_IMPORT_DESCRIPTOR   10006928     msvcprt:MSVCP80.dll
 0003:00000004       ??_R0?AVBaseExc@Iex@@@8    10008004     IexBaseExc.obj
 0003:00000020       ??_R0?AV?$basic_string@DU?$char_traits@D@std@@V?$allocator@D@2@@std@@@8 10008020     IexBaseExc.obj
 0003:0000006c       ??_R0?AV?$_String_val@DV?$allocator@D@std@@@std@@@8 1000806c     IexBaseExc.obj
 0003:000000a4       ??_R0?AV_String_base@std@@@8 100080a4     IexBaseExc.obj
 0003:000000c4       ??_R0?AU_Container_base@std@@@8 100080c4     IexBaseExc.obj
 0003:000000e8       ??_R0?AVexception@std@@@8  100080e8     IexBaseExc.obj
 0003:00000108       ??_R0?AVEpermExc@Iex@@@8   10008108     IexThrowErrnoExc.obj
 0003:00000124       ??_R0?AVErrnoExc@Iex@@@8   10008124     IexThrowErrnoExc.obj
 0003:00000140       ??_R0?AVEnoentExc@Iex@@@8  10008140     IexThrowErrnoExc.obj
 0003:0000015c       ??_R0?AVEsrchExc@Iex@@@8   1000815c     IexThrowErrnoExc.obj
 0003:00000178       ??_R0?AVEintrExc@Iex@@@8   10008178     IexThrowErrnoExc.obj
 0003:00000194       ??_R0?AVEioExc@Iex@@@8     10008194     IexThrowErrnoExc.obj
 0003:000001b0       ??_R0?AVEnxioExc@Iex@@@8   100081b0     IexThrowErrnoExc.obj
 0003:000001cc       ??_R0?AVE2bigExc@Iex@@@8   100081cc     IexThrowErrnoExc.obj
 0003:000001e8       ??_R0?AVEnoexecExc@Iex@@@8 100081e8     IexThrowErrnoExc.obj
 0003:00000208       ??_R0?AVEbadfExc@Iex@@@8   10008208     IexThrowErrnoExc.obj
 0003:00000224       ??_R0?AVEchildExc@Iex@@@8  10008224     IexThrowErrnoExc.obj
 0003:00000240       ??_R0?AVEagainExc@Iex@@@8  10008240     IexThrowErrnoExc.obj
 0003:0000025c       ??_R0?AVEnomemExc@Iex@@@8  1000825c     IexThrowErrnoExc.obj
 0003:00000278       ??_R0?AVEaccesExc@Iex@@@8  10008278     IexThrowErrnoExc.obj
 0003:00000294       ??_R0?AVEfaultExc@Iex@@@8  10008294     IexThrowErrnoExc.obj
 0003:000002b0       ??_R0?AVEbusyExc@Iex@@@8   100082b0     IexThrowErrnoExc.obj
 0003:000002cc       ??_R0?AVEexistExc@Iex@@@8  100082cc     IexThrowErrnoExc.obj
 0003:000002e8       ??_R0?AVExdevExc@Iex@@@8   100082e8     IexThrowErrnoExc.obj
 0003:00000304       ??_R0?AVEnodevExc@Iex@@@8  10008304     IexThrowErrnoExc.obj
 0003:00000320       ??_R0?AVEnotdirExc@Iex@@@8 10008320     IexThrowErrnoExc.obj
 0003:00000340       ??_R0?AVEisdirExc@Iex@@@8  10008340     IexThrowErrnoExc.obj
 0003:0000035c       ??_R0?AVEinvalExc@Iex@@@8  1000835c     IexThrowErrnoExc.obj
 0003:00000378       ??_R0?AVEnfileExc@Iex@@@8  10008378     IexThrowErrnoExc.obj
 0003:00000394       ??_R0?AVEmfileExc@Iex@@@8  10008394     IexThrowErrnoExc.obj
 0003:000003b0       ??_R0?AVEnottyExc@Iex@@@8  100083b0     IexThrowErrnoExc.obj
 0003:000003cc       ??_R0?AVEfbigExc@Iex@@@8   100083cc     IexThrowErrnoExc.obj
 0003:000003e8       ??_R0?AVEnospcExc@Iex@@@8  100083e8     IexThrowErrnoExc.obj
 0003:00000404       ??_R0?AVEspipeExc@Iex@@@8  10008404     IexThrowErrnoExc.obj
 0003:00000420       ??_R0?AVErofsExc@Iex@@@8   10008420     IexThrowErrnoExc.obj
 0003:0000043c       ??_R0?AVEmlinkExc@Iex@@@8  1000843c     IexThrowErrnoExc.obj
 0003:00000458       ??_R0?AVEpipeExc@Iex@@@8   10008458     IexThrowErrnoExc.obj
 0003:00000474       ??_R0?AVEdomExc@Iex@@@8    10008474     IexThrowErrnoExc.obj
 0003:00000490       ??_R0?AVErangeExc@Iex@@@8  10008490     IexThrowErrnoExc.obj
 0003:000004ac       ??_R0?AVEdeadlkExc@Iex@@@8 100084ac     IexThrowErrnoExc.obj
 0003:000004cc       ??_R0?AVEnolckExc@Iex@@@8  100084cc     IexThrowErrnoExc.obj
 0003:000004e8       ??_R0?AVEnametoolongExc@Iex@@@8 100084e8     IexThrowErrnoExc.obj
 0003:0000050c       ??_R0?AVEilseqExc@Iex@@@8  1000850c     IexThrowErrnoExc.obj
 0003:00000528       ??_R0?AVEnosysExc@Iex@@@8  10008528     IexThrowErrnoExc.obj
 0003:00000544       ??_R0?AVEnotemptyExc@Iex@@@8 10008544     IexThrowErrnoExc.obj
 0003:00000564       ??_R0?AVtype_info@@@8      10008564     MSVCRT:ti_inst.obj
 0003:0000057c       ___security_cookie         1000857c     MSVCRT:gs_cookie.obj
 0003:00000580       ___security_cookie_complement 10008580     MSVCRT:gs_cookie.obj
 0003:00000598       ?_RTC_ErrorLevels@@3PAHA   10008598     MSVCRT:error.obj
 0003:000005c4       ___native_dllmain_reason   100085c4     MSVCRT:natstart.obj
 0003:000005c8       ___native_vcclrit_reason   100085c8     MSVCRT:natstart.obj
 0003:000005d0       ?currentStackTracer@?A0x883d44e9@Iex@@3P6A?AV?$basic_string@DU?$char_traits@D@std@@V?$allocator@D@2@@std@@XZA 100085d0     IexBaseExc.obj
 0003:000005e0       ?wsprintffp@@3P6AHPADPBDZZA 100085e0     MSVCRT:error.obj
 0003:0000090c       ?__type_info_root_node@@3U__type_info_node@@A 1000890c     MSVCRT:tncleanup.obj
 0003:00000920       __adjust_fdiv              10008920     <common>
 0003:00000924       ___native_startup_state    10008924     <common>
 0003:00000928       ___native_startup_lock     10008928     <common>
 0003:0000092c       ___onexitend               1000892c     <common>
 0003:00000930       ___onexitbegin             10008930     <common>
 0003:00000934       ___dyn_tls_init_callback   10008934     <common>

 entry point at        0001:00001dac

 Static symbols

 0001:00001aaa       _pre_c_init                10002aaa f   MSVCRT:crtdll.obj
 0001:00001c96       ___DllMainCRTStartup       10002c96 f   MSVCRT:crtdll.obj
 0001:00001dd9       ?DebuggerProbe@@YAHK@Z     10002dd9 f   MSVCRT:error.obj
 0001:00001e29       ?DebuggerRuntime@@YAHKHPAXPB_W@Z 10002e29 f   MSVCRT:error.obj
 0001:00001e8b       ?failwithmessage@@YAXPAXHHPBD@Z 10002e8b f   MSVCRT:error.obj
 0001:00002698       ?GetPdbDll@@YAPAUHINSTANCE__@@XZ 10003698 f   MSVCRT:pdblkup.obj
 0001:00002aa0       __unwindfunclet$?assign@BaseExc@Iex@@QAEAAV12@AAV?$basic_stringstream@DU?$char_traits@D@std@@V?$allocator@D@2@@std@@@Z$0 10003aa0 f   IexBaseExc.obj
 0001:00002ab2       __ehhandler$?assign@BaseExc@Iex@@QAEAAV12@AAV?$basic_stringstream@DU?$char_traits@D@std@@V?$allocator@D@2@@std@@@Z 10003ab2 f   IexBaseExc.obj
 0001:00002acd       __unwindfunclet$?append@BaseExc@Iex@@QAEAAV12@AAV?$basic_stringstream@DU?$char_traits@D@std@@V?$allocator@D@2@@std@@@Z$0 10003acd f   IexBaseExc.obj
 0001:00002adf       __ehhandler$?append@BaseExc@Iex@@QAEAAV12@AAV?$basic_stringstream@DU?$char_traits@D@std@@V?$allocator@D@2@@std@@@Z 10003adf f   IexBaseExc.obj
 0001:00002b00       __unwindfunclet$?throwErrnoExc@Iex@@YAXABV?$basic_string@DU?$char_traits@D@std@@V?$allocator@D@2@@std@@H@Z$0 10003b00 f   IexThrowErrnoExc.obj
 0001:00002b12       __ehhandler$?throwErrnoExc@Iex@@YAXABV?$basic_string@DU?$char_traits@D@std@@V?$allocator@D@2@@std@@H@Z 10003b12 f   IexThrowErrnoExc.obj
